:1000000010308A0000280000FF00030E8301A100C9
:100010000A08A0008A010408A2007708A300780853
:10002000A4007908A5007A08A6007B08A70083131E
:1000300083128B1D1D280B1846280B1E21288B1898
:1000400049288C308400801E27288C1A4C288C303C
:100050008400001C2D280C184F288C308400801C34
:1000600033288C185228220884002308F70024081B
:10007000F8002508F9002608FA002708FB002008E8
:100080008A00210E8300FF0E7F0E09008A110A12DA
:10009000B6298A110A120D298A110A12102A8A1108
:1000A0000A12452A8A110A12342A0A108A100A11E1
:1000B000820728340C34013406340A108A100A11DD
:1000C000820745344C343D3400340A108A100A113A
:1000D00082072D3400340A108A100A118207203456
:1000E00000340A108A100A11820754344834453407
:1000F0004E3420345034553453344834203427346B
:100100005034413452344B34273400340A108A10AE
:100110000A1182074F34463446345334453454343C
:100120002034573445345334543400340A108A1080
:100130000A1182075234453446344534523445342A
:100140004E3443344534203400340A108A100A11E6
:100150008207533445345434203441345A344934BA
:100160004D345534543420343E34203400340A1095
:100170008A100A11820753344534543420344534EC
:100180004C34203454344F3420345A3445345234AF
:100190004F3420342034203400340A108A100A11DD
:1001A000820741345A3400340A108A100A11820737
:1001B00045344C3400340A108A100A118207543432
:1001C00000340A108A100A1182070C3400340A1015
:1001D0008A100A11820744344534533459344E345A
:1001E000433420344D344F3454344F34523400347B
:1001F0000000000000000A148A100A11023E0318D1
:100200008A0A82005234413445344C34203452340A
:100210004F3454344F345234003483160510831253
:10022000051083168510831285108316851183129D
:10023000851183160511831205110B138B138B1B6C
:100240001E291030F700F70B232900003008031790
:10025000A800A90104308D0028088C0083168C1397
:100260000C15831203130B08F7008B138316031767
:1002700055308D00AA308D008C148C183D290C113E
:100280007708831203138B041030F700F70B46290D
:100290000000053003178D0003132F0803178C008F
:1002A00083168C130C15831203130B08F7008B13A2
:1002B0008316031755308D00AA308D008C148C18CE
:1002C0005F290C117708831203138B041030F70099
:1002D000F70B6829000032080317A800A9010230B3
:1002E0008D0028088C0083168C130C1583120313C1
:1002F0000B08F7008B138316031755308D00AA30B7
:100300008D008C148C1882290C117708831203132A
:100310008B041030F700F70B8B2900000330031714
:100320008D000313310803178C0083168C130C15F2
:10033000831203130B08F7008B1383160317553032
:100340008D00AA308D008C148C18A4290C1177080C
:10035000831203138B041030F700F70BAD29000054
:10036000630063008B108A110A12332806083039A3
:1003700051060317A80003130608D1000317A81E8F
:10038000D4290313C1080319C9290130AF07031881
:10039000B00AC2080319D2290130AF020030031C91
:1003A0000130B002C3010317281EE9290313BF0857
:1003B0000319DE290130B1070318B20AC008031976
:1003C000E7290130B1020030031C0130B202C30141
:1003D0000317AA01A9012A08273C031CFE29031DB3
:1003E000F52929080F3C031CFE2929080319AA0333
:1003F000A9030230A9070318AA0AEB2903130B105B
:100400008A110A1233288C1E032A1808A8001A0819
:10041000F800A81C0D2A181218168A110A12112A9F
:10042000032A78080317A80028081F3C031C1C2A6D
:1004300028080D3C031D2F2A03134C08FA004B0813
:10044000CB0A0319CC0A0317A9007A08AA00A03026
:100450002907840083132A188317280880000313B0
:100460008C128A110A1233285708033C031C412AB4
:10047000031D3E2A5608F13C031C412AD60A0319E3
:10048000D70A8C108A110A123328C30A0C108A1159
:100490000A1233281F3084008317000803195D2ACD
:1004A0000630F800F701F70B532AF80B522A7B307D
:1004B000F700F70B592A800B502A00340317260E39
:1004C000F039F7000F3003130805770488000000A7
:1004D00008140330F700F70B6B2A0810003488105B
:1004E000F0308316880083120815000008140000FD
:1004F0000808080E0F390317A600031308100000A0
:100500000814822A832A00000808080E0F390317EE
:10051000A500031308100030831688008312031708
:10052000260EF700F030F70577082504F800780864
:10053000A500A51F9D2A0313702A2318A22A0313BE
:1005400088100317231CA72A03138814031700001D
:1005500003130811000008100317240EA5000F3024
:10056000A5052508A60003135E22031724080F39EA
:10057000A500A60003135E22003400308316880015
:1005800083128810081108100F3003179F000313FF
:100590004A2201308316DC005C08033C031CDE2A7F
:1005A000033083120317A60003135E2205300317DE
:1005B0009F0003134A228316DC0ACC2A02308312DE
:1005C0000317A60003135E228316DC015C08033CBC
:1005D000031CFD2A5C08831255208316DD0083125C
:1005E0000317A301831603135D0883120317A400E6
:1005F00003136F228316DC0AE62A83128A110A1675
:10060000DB280317200B052B082B4030A100092BFA
:10061000A10101301F02A10721088038A200A30117
:100620002208A40003136F22003403171E080C3A9B
:1006300003130319222B063A03192E2B023A03192E
:10064000362B3D2B0317A3010130A40003136F22A7
:10065000023003179F0003134A22452B0130031772
:100660009F000230A00003130123452B0317A301B1
:100670001030A40003136F22452B01300317A30091
:100680001E08A40003136F22452B003403179D019D
:1006900004089C001D10831B1D14160EF0389800D2
:1006A0009807E23E9900323E9B0016080F399907E1
:1006B00099079B07E93E9A009A079A07150E0F398A
:1006C0009A079B079A0D9B0D9B099B0D15080F39E7
:1006D0009B07980D073097000A309B079A03031C6D
:1006E0006D2B9A079903031C712B99079803031C20
:1006F000752B98079703031C792B173084008317F9
:1007000007301C051C1384071B30040203191C1737
:100710000008F700031D942B1C1B942B1C1AA82BFC
:100720009C19942B2030972B9C151C123030F70706
:100730009601040895001610831B161477089E0076
:100740000313152303171508840083131618831742
:10075000840A1C1F842B03130034F701F80183164D
:10076000620803106318F707F70CF80CE318F70793
:10077000F70CF80C6319F707F70CF80CE319F707F7
:10078000F70CF80C631AF707F70CF80CE31AF707E5
:10079000F70CF80C631BF707F70CF80CE31BF707D3
:1007A000F70CF80C831200340B138B138B1BD52B17
:1007B00083166608E700E8016408831203178D00BA
:1007C000831603136608831203178C0083168C1399
:1007D0000C15831203130B08F7008B1383160317F2
:1007E00055308D00AA308D008C148C18F52B0C110F
:1007F0007708831203138B04013083166407E70024
:10080000831203178D0083160313650883120317E1
:100810008C0083168C130C15831203130B08F7003E
:100820008B138316031755308D00AA308D008C145E
:100830008C18182C0C117708831203138B04C0300A
:100840008B0400348316DC01DD01E001E101831239
:100850000B138B138B1B292C013003179F000230C5
:10086000A000031301238316E201620883127120A2
:1008700000380319452C8316E20A831203179E00E1
:10088000031315238316352C8312013003179F00A1
:10089000A000031301238316E2016208831286205D
:1008A000003803195D2C8316E20A831203179E0099
:1008B0000313152383164D2C83123D3003179E001E
:1008C0000313152302308400831661088312031773
:1008D0009600831603136008831203179500031311
:1008E000462304308316E200FA30831203179F0078
:1008F00003134A228316E20B742C09148312091C79
:10090000052DE8308316DE000130DF008312071862
:10091000C42C871DC42C8316E108031D972C600886
:10092000B33C031C972C0130E0070318E10A5E0872
:10093000831203179F0003134A228316DF0A5E08FF
:100940001E3C0318AC2C1430E2005F08E300831255
:10095000AD2378088316DE020D30831203179F0043
:100960000130A000031301230230840083166108C4
:10097000831203179600831603136008831203176C
:10098000950003134623872C8719022D071C022D7F
:100990008316E008031DCF2CE1080319D52C013084
:1009A000E0020030031C0130E1025E0883120317ED
:1009B0009F0003134A228316DF0A5E081E3C0318B9
:1009C000EA2C1430E2005F08E3008312AD237808BC
:1009D0008316DE020D30831203179F000130A00042
:1009E0000313012302308400831661088312031766
:1009F00096008316031360088312031795000313F0
:100A00004623C42C83167D2C831206308316E40003
:100A10006108E6006008E5008312D42304308316E1
:100A2000E200FA30831203179F0003134A22831651
:100A3000E20B112D0130831203179F000230A0003A
:100A4000031301238316E201620883127120003828
:100A50000319342D8316E20A831203179E00031331
:100A600015238316242D8312013003179F00A00045
:100A7000031301238316E2016208831296200038D3
:100A800003194C2D8316E20A831203179E000313E9
:100A9000152383163C2D8312413003179E00031348
:100AA00015235A3003179E00031315233D300317F7
:100AB0009E00031315230230840083165D08831201
:100AC00003179600831603135C088312031795001F
:100AD00003134623831609148312091C122EE830CF
:100AE0008316DE000130DF0083120718C42D871D36
:100AF000C42D83165D08013C031C882D031D842D25
:100B00005C08673C031C882D0130DC070318DD0AF4
:100B10005E08831203179F0003134A228316DF0A1D
:100B20005E081E3C03189D2D1430E2005F08E300B0
:100B30008312AD2378088316DE020B30831203176D
:100B40009F000130A00003130123413003179E00D2
:100B5000031315235A3003179E00031315233D304A
:100B600003179E00031315230230840083165D08CB
:100B7000831203179600831603135C08831203176E
:100B8000950003134623752D8719112E071C112E6E
:100B90008316DC08031DCF2DDD080319D52D013088
:100BA000DC020030031C0130DD025E0883120317F3
:100BB0009F0003134A228316DF0A5E081E3C0318B7
:100BC000EA2D1430E2005F08E3008312AD237808B9
:100BD0008316DE020B30831203179F000130A00042
:100BE00003130123413003179E00031315235A30CA
:100BF00003179E00031315233D3003179E000313B4
:100C000015230230840083165D08831203179600B3
:100C1000831603135C0883120317950003134623FE
:100C2000C42D6A2D013003179F00A0000313012378
:100C30008316E20162088312A520003803192A2EC8
:100C40008316E20A831203179E00031315238316EB
:100C50001A2E83120230840083165D088312031754
:100C60009600831603135C08831203179500031381
:100C7000462304308316E200C830831203179F0016
:100C800003134A228316E20B3C2E09148312091C1B
:100C9000652E871D4D2E07185A2E0718532E8316C2
:100CA0000511831205158719592E83168511831294
:100CB0008515492E8316851183128511831605111A
:100CC000831205118316452E8312031083165C0DC3
:100CD000E2005D0DE30083124D0883166207831264
:100CE000AF00831663088312B0004E0803184E0F3E
:100CF000B00703108316600DF900610DFA00790842
:100D000083122F078316E200831230088316E30054
:100D10007A0803187A0FE3070430E4006308E6005A
:100D20006208E5008312D42304308316E200C83041
:100D3000831203179F0003134A228316E20B972E98
:100D40000130831203179F00A000031301238316B1
:100D5000E20162088312B72000380319B92E831606
:100D6000E20A831203179E00031315238316A92E8C
:100D70008312013003179F000230A00003130123E8
:100D80008316E20162088312712000380319D22E03
:100D90008316E20A831203179E000313152383169A
:100DA000C22E8312831609148312091CF12E871E8A
:100DB000DB2E071AE82E871AE12E83168510831280
:100DC0008514071AE72E8316051083120514D72EF3
:100DD0008316051083120510831685108312851063
:100DE000D22E14304F078316E20083125008831668
:100DF000E3000318E30A0230E4006308E600620837
:100E0000E5008312D42304308316E200FA30831203
:100E100003179F0003134A228316E20B062F8A0151
:100E2000831200288A110A16F9288316DE01DF01D1
:100E30005C08831203178D0083168C130C14831225
:100E40000C0883160313DF01DE000530831203173D
:100E50009F0003134A2283165E08E100E00101307F
:100E60005C07E2005D08E3000318E30A62088312EE
:100E700003178D0083168C130C1483120C08831631
:100E800003136004DE006108DF005E08F8005F08FD
:100E9000F9008312003483166508FA0064088400A0
:100EA00083137A18831780080319962F6508E900C1
:100EB0006408E8006708EB006608EA006B08FA00BF
:100EC0006A08840083137A18831780080319832F14
:100ED0006908FA006808840083137A1883170008E9
:100EE000EC006B08FA006A08840083137A188317F1
:100EF00000086C02031D832FE80A0319E90AEA0AB5
:100F00000319EB0A5E2F6B08FA006A08840083134A
:100F10007A1883178008031D922F6408F80065086B
:100F2000F900992FE40A0319E50A4C2F0030F80064
:100F3000F90083120034103003179F00F701FA0103
:100F40009C0C9B0C031CAA2F1D08F7070318FA0A18
:100F50001E08FA07FA0CF70CF90CF80C9F0BA02FDF
:100F600003138A150A127728F801F901F701FA012B
:100F700003171708031DBF2F16080319D92F1030A8
:100F800098000310940D950DF70DFA0D17087A02CD
:100F9000031DCC2F16087702031CD52F1608F70265
:100FA000031CFA031708FA020314F80DF90D980B45
:060FB000C12F0313003401
:101000000317990197010A3098009601950113087A
:101010001404031D0F280030F800F90008291908EE
:10102000990A1307840083131418831700089A0081
:101030001A082D3C031D2828013097001908990A29
:101040001307840083131418831700089A003528A7
:101050001A082B3C031D35281908990A1307840028
:1010600083131418831700089A001A082F3C0318DA
:10107000F9281A08393C031CF9281A08303C031DCA
:1010800061281908130784008313141883170008B4
:10109000783C031955281908130784008313141882
:1010A00083170008583C031D612810309800990AE6
:1010B0001908990A1307840083131418831700086A
:1010C0009A0018080A3C031D90281A082F3C0318A0
:1010D0008F281A08393C031C8F289C010A309B007A
:1010E00016089E0015089D008A1103139B2F8A1570
:1010F000790803179C0078089B0030301A021B0700
:1011000095001C0896000318960A1908990A1307F7
:10111000840083131418831700089A006528F9289F
:101120001808103C031DF9281A08603C03189F2872
:101130001A087A3C031C9F281A08DF39A0281A08CD
:101140009A001A082F3C0318A9281A08393C0318DA
:10115000B1281A08403C0318F9281A08463C031C19
:10116000F9281A082F3C0318CE281A08393C031C0A
:10117000CE28150D9B00160D9C009B0D9C0D9B0D04
:101180009C0D9B0D9C0DF0309B0530301A021B0707
:1011900095001C0896000318960AE328150D9B007D
:1011A000160D9C009B0D9C0D9B0D9C0D9B0D9C0D8D
:1011B000F0309B0541301A020A3E1B0795001C08BF
:1011C00096000318960A1908990A130784008313D6
:1011D0001418831700089A00603C0318F6281A08B0
:1011E0007A3C031CF6281A08DF39F7281A089A00F7
:1011F000A12818080A3C031D0429170B0429950986
:101200009609950A0319960A1508F8001608F900B8
:10121000031300348316E601EF01831203179001D4
:101220000430F800E730840083138001840AF80B4F
:1012300015290430F800EB30840083138001840A00
:10124000F80B1E2983160313E401E501831203172B
:101250009201A03091001208940011089300140824
:10126000FA001308840083137A188317800803197F
:101270003D29930A0319940A2F2911081302F70034
:101280001408FA001208031C120FFA027708F8007B
:101290007A08F9007908FA007808FA08031D582935
:1012A00078088316031364020318F22983120317C4
:1012B000A0308316031364078400831300082E3CB8
:1012C000031D6A29EF010130831203179000EE29F4
:1012D00083160313A0306407840083130008203CA6
:1012E000031D7929EF01831203179001EE2983165C
:1012F0000313A03064078400831300082F3C0318F5
:101300008929A0306407840083130008393C03183E
:101310008E2983120317EE298316031383120317F2
:10132000100B9329EE2983160313EF08031D9C2944
:10133000E501E60A0130EF006608013A831203195D
:10134000A529033A0319C729EA29E7308316650757
:10135000F800FA010318FA0A7808831203179100BB
:101360007A089200A0308316031364078400831365
:1013700000088312031793001108840083131218C6
:1013800083171308800083160313E50AEC29EB305A
:1013900083166507F800FA010318FA0A7808831221
:1013A000031791007A089200A03083160313640794
:1013B000840083130008831203179300110884002C
:1013C0008313121883171308800083160313E50A8A
:1013D000EC2983128316EC29831203178316031357
:1013E000E40A2629831203179401E73093000313BC
:1013F000002079080317920078089100921B172AA1
:101400009401E73093000313002079080317940038
:1014100078089300941B1A2A1408003C03181A2A0F
:10142000FF3A031D172A1308683C03181A2A0030D4
:10143000F800522A9401EB3093000313002079083E
:101440000317920078089100921B392A9401EB301F
:101450009300031300207908031794007808930081
:10146000941B3C2A9408031D392A13085A3C03187C
:101470003C2A0030F800522A9401E730930003130D
:1014800000207908B6007808B50003179401EB3006
:101490009300031300207908B4007808B3000130EA
:1014A000F800031703138A150A12932C8316ED0113
:1014B000EE010130831203179F008316031368089F
:1014C00083120317A0008A11031301238A155808F9
:1014D000683C031790000130910003135908031C66
:1014E000590F732A762A03179102031383166B0888
:1014F0008312031710079200110893008316031339
:101500006C0803186C0F852A8A2A83120317930725
:10151000831603138312031713089500120894000F
:1015200001309700683096008A110313B4278A159A
:101530007708031793007A08940041309E008A11BF
:10154000031315238A155A3003179E008A110313BB
:1015500015238A153D3003179E008A1103131523A6
:101560008A150230840003171408960013089500AA
:101570008A11031346238A15DF3003179E008A1150
:10158000031315238A1583166A088312031795001F
:101590008316031369088312031794000130970020
:1015A000683096008A110313B4278A1577085E3EC7
:1015B0008316ED007A08EE00013003180230EE07C2
:1015C0000830831203179F008316031368088312E1
:1015D0000317A0008A11031301238A150317900132
:1015E00010088A1103135D208A1500380319022B95
:1015F0000317900A9E008A11031315238A150317F7
:10160000F02A031383166E088312031795008316BE
:1016100003136D088312031794000130970068309C
:1016200096008A110313B4278A15770803179000D0
:101630007A0891009108031D212B1008C83C03185B
:10164000452B831603136D08683CED006E08031CE0
:101650006E0F2C2B01302D2B013CEE008312031753
:10166000900110088A11031365208A1500380319A8
:10167000432B0317900A9E008A11031315238A1522
:101680000317312B0313582B0317900110088A11ED
:1016900003136B208A1500380319582B0317900A7F
:1016A0009E008A11031315238A150317462B031373
:1016B00083166E08831203179500831603136D08B3
:1016C00083120317940001309700683096008A1146
:1016D0000313B4278A157708031790007A0891003E
:1016E0000230840011089600100895008A11031337
:1016F00046238A15DF3003179E008A110313152332
:101700008A1500344E083002031CA62B031D8C2BB7
:101710004D082F02031CA62B4D082F028316E40050
:10172000831230088316E50083124E08031C4E0F07
:101730009A2B9D2B8316E502831203108316650CEA
:101740008312BA008316640C8312B90030084E026B
:10175000031CCA2B031DB02B4D082F020318CA2BE4
:101760002F084D028316E40083124E088316E5000D
:1017700083123008031C300FBE2BC12B8316E502E9
:10178000831203108316650C8312BA008316640C4F
:101790008312B90050083202031CEE2B031DD42B18
:1017A0004F083102031CEE2B4F0831028316E40070
:1017B000831232088316E50083125008031C500F71
:1017C000E22BE52B8316E502831203108316650CCA
:1017D0008312B8008316640C8312B70032085002DB
:1017E000031C122C031DF82B4F0831020318122C76
:1017F00031084F028316E400831250088316E50077
:1018000083123208031C320F062C092C8316E502C2
:10181000831203108316650C8312B8008316640CC0
:101820008312B700003401304B028316E4008312A8
:101830004C088316E5000030031C0130E502A0309F
:101840006407840083136518831700080D3C031D8B
:10185000AC2D013083124B028316E40083124C0836
:101860008316E5000030031C0130E502A030640758
:1018700084008313651883178001E401E501DC30DF
:10188000840083136408840765088A118312CD20BD
:101890008A15800000380319522C8316E50AE40AE1
:1018A0003F2C83128316E401E501E03084008313AA
:1018B0006408840765088A118312D4208A15800081
:1018C00000380319682C8316E50AE40A552C8312A4
:1018D0008316E501A030E400E701DC30E6008A1160
:1018E00083124B278A15780879040319862C8316EE
:1018F000E501A030E400E701E030E6008A11831240
:101900004B278A1578087904031D922C831620082A
:101910004D3C031D8D2C8312922C2008573C031D37
:10192000A72D83120A29F8080319A82DD701D6017B
:101930000A3033078316E400831234088316E50067
:101940000318E50A8312580835078316E600831248
:1019500036088316E700831259080318590FB12C73
:10196000B42C8316E707831201308316E80065085C
:10197000EA006408E9006708EC006608EB008312DF
:101980005622822301303907F8003A08FA0003187A
:10199000FA0A7A083602031CD32C031D002D3508E1
:1019A0007802031C002D0A3035078316E4008312E9
:1019B00036088316E5000318E50A0A308312390752
:1019C0008316E60083123A088316E7000318E70A35
:1019D00001306602F7006708FA000030031C01308E
:1019E000FA027708F80065087A02031C0A2D031929
:1019F000FB2C8312002D7808640203180A2D831231
:101A00000130CA00D501D4013A08D3003908D20008
:101A10000C2D83168312CA010A3033078316E400A3
:101A2000831234088316E5000318E50A0130831297
:101A30003707F8003808FA000318FA0A7A088316FC
:101A40006502031C292D031D542D64087802031C14
:101A5000542D1E30831233078316E6008312340898
:101A60008316E7000318E70A14308312370783163A
:101A7000E800831238088316E9000318E90A0130E8
:101A80006802F7006908FA000030031C0130FA020E
:101A90007708F80067087A02031C592D031D542D9E
:101AA000780866020318592D01308312C9005B2D96
:101AB00083168312C901103003179F000130A00064
:101AC0008A11031301238A158316E40164088A111D
:101AD0008312DB208A15003803197A2D8316E40A55
:101AE000831203179E008A11031315238A15831688
:101AF000662D831202308316E400C8308312031768
:101B00009F008A1103134A228A158316E40B7D2D48
:101B10001030831203179F000130A0008A110313B5
:101B200001238A158316E40164088A1183126B204D
:101B30008A1500380319A82D8316E40A83120317A7
:101B40009E008A11031315238A158316942D831280
:101B5000CC01CB018316A00183128A110A16EE294B
:101B60004308283C0318F32D831685118312851131
:101B7000831605118312051107118316DC015C0819
:101B80008A118312E1208A1500380319D32D831698
:101B9000DC0A831203179E008A11031315238A158A
:101BA0008316BF2D8312033003179F000130A0005E
:101BB0008A11031301238A158316DC015C088A113C
:101BC0008312E7208A1500380319F22D8316DC0AE8
:101BD000831203179E008A11031315238A15831697
:101BE000DE2D83126300003483168C120C148312D2
:101BF0004A0B052E83168511831285118316051154
:101C0000831205110230CA00FA2E490B122E8316D8
:101C1000851083128510831605108312051002307B
:101C2000C900FA2E871A4A2E071E4A2E871A492EF5
:101C3000071E492EB808031D492E3708633C031CB4
:101C4000492E83168510831285140130BF00C00110
:101C500082230C3003179F000130A0008A11031368
:101C600001238A1502308316E80083123808831690
:101C7000EA00831237088316E90083123A088316B4
:101C8000EC00831239088316EB0083125622B0252C
:101C9000162E7C2E071A7C2E871E7C2EB708031D5D
:101CA000542EB80803197C2E8316051083120514D0
:101CB000BF010130C00082230C3003179F000130A8
:101CC000A0008A11031301238A1502308316E8004D
:101CD000831238088316EA00831237088316E90056
:101CE00083123A088316EC00831239088316EB003E
:101CF00083125622B0254A2E831685108312851032
:101D000083160510831205100230C9000718C22E71
:101D1000871DC22E0718C12E871DC12E3A08013C0F
:101D2000031CC12E031D982E3908C13C031CC12E73
:101D3000071583160511831205150130C100C20174
:101D400082230C3003179F000130A0008A11031377
:101D500001238A1502308316E8008312380883169F
:101D6000EA00831237088316E90083123A088316C3
:101D7000EC00831239088316EB0083125622B0253B
:101D80008A2EEC2E8719EC2E071CEC2EB908031DA9
:101D9000CC2EBA080319EC2E071583168511831271
:101DA0008515C1010130C200822302308316E8008C
:101DB000831238088316EA00831237088316E90075
:101DC00083123A088316EC00831239088316EB005D
:101DD00083125622B025C22E0711831605118312D5
:101DE000051183168511831285110230CA008316EE
:0A1DF0008C1683128A110A16762C55
:10200000840183131F308305FF3083169900A230AB
:10201000980090308312980083161F149F141F1588
:102020009F1107309C008312A801A901AA01AF01EA
:10203000B001B101B201B301B401B501B601B701FC
:10204000B801B901BA01BB01BC01BD01BE01BF01AC
:10205000C001C101C201C3018316A001A101A201F7
:10206000A301A401A501A601A701A801A901AA0134
:10207000AB01AC01AD01AE01AF01B001B101B201E4
:10208000B301B401B501B601B701B801B901BA0194
:10209000BB01BC01BD01BE01BF01C001C101C20144
:1020A000C301C401C501C601C701C801C901CA01F4
:1020B000CB01CC01CD01CE01CF01D001D101D201A4
:1020C000D301D401D501D601D701D801D901DA0154
:1020D000DB018312C401C501C601C701C801C901E2
:1020E000CA01CB01CC01E830CD000330CE00E8308E
:1020F000CF000330D000D101D201D301D401D501EA
:102100002030D6000330D700D801D9010030831623
:102110008500FF308600B93087000914891409153D
:1021200085108312851083160510831205108316FF
:10213000851183128511831605118312051107116C
:1021400087140730F700F71DAE2807308101813072
:10215000840083130008C0390F3880006400813088
:1021600084000008C03977048000B53090007830D2
:10217000F80006389200FF30831692001F149F1457
:102180001F159F1183121F108316091283129412B8
:102190000030940083169400011383120B1603176A
:1021A0008B15831603138C160C108C14C0308312FD
:1021B0008B040A12BD2A0A168316DC015C080A1277
:1021C0008312E1200A1600380319F2288316DC0A6C
:1021D000831203179E000A12031315230A1683168F
:1021E000DE2883128316091583120919FA280A12A8
:1021F000222C0A168316DD010230DC000A1283123B
:1022000015270A167908B2007808B1005008320282
:10221000031C2A29031D10294F083102031C2A29F7
:102220004F0831028316DC00831232088316DD006A
:1022300083125008031C500F1E2921298316DD022A
:102240008312031083165D0C8312B80083165C0C96
:102250008312B70032085002031C4E29031D342993
:102260004F08310203184E2931084F028316DC0053
:10227000831250088316DD0083123208031C320FCC
:10228000422945298316DD028312031083165D0C53
:102290008312B80083165C0C8312B7003808B400B0
:1022A0003708B3008316DD010430DC000A12831204
:1022B00015270A167908B0007808AF004E083002DA
:1022C000031C8229031D68294D082F02031C822943
:1022D0004D082F028316DC00831230088316DD00C0
:1022E00083124E08031C4E0F762979298316DD02CE
:1022F0008312031083165D0C8312BA0083165C0CE4
:102300008312B90030084E02031CA629031D8C2934
:102310004D082F020318A6292F084D028316DC0052
:1023200083124E088316DD0083123008031C300F21
:102330009A299D298316DD028312031083165D0CF2
:102340008312BA0083165C0C8312B9003A08B600F7
:102350003908B5008316DD010630DC000A1283124D
:1023600015270A167908D9007808D8008316DC01E9
:102370005C080A128312E1200A1600380319CC29DE
:102380008316DC0A831203179E000A120313152317
:102390000A168316B8298312043003179F000130F0
:1023A000A0000A12031301230A168316DC015C083D
:1023B0000A128312F8200A1600380319EB29831633
:1023C000DC0A831203179E000A12031315230A1650
:1023D0008316D72983120A128A15132C0A168A111A
:1023E0004A0B2A2B3A083602031C0F2A031DFC292C
:1023F0003508390203180F2A39083502BD0036089E
:10240000BE003A08031C3A0FBE0252083902BB0054
:102410003A08BC005308031C530FBC02212A35089C
:102420003902BD003A08BE003608031C360FBE0252
:1024300039085202BB005308BC003A08031C3A0F8B
:10244000BC02BC08031D282A3B08053C03182F2AA0
:10245000BE08031D312A3D08053C031C312A071123
:10246000322A071583168C128312580835078316F3
:10247000DC00831236088316DD0083125908031826
:10248000590F432A462A8316DD0783120310831649
:102490005C0DDE005D0DDF0083124D0883165E07C4
:1024A0008312C70083165F088312C8004E08031802
:1024B0004E0FC8070A128A1582230A168A11C2080B
:1024C00003199B2A30084802031C9B2A031D6C2A0F
:1024D0002F084702031C9B2A83168511831285113E
:1024E00002308316E800831238088316EA0083124C
:1024F00037088316E90083123A088316EC0083122A
:1025000039088316EB000A128A15831256220A161E
:102510008A1102308316DC00FA30831203179F0001
:102520000A1203134A220A168316DC0B8C2A023085
:102530008312CA00272BC1080319D72A4808300282
:10254000031CD72A031DA82A47082F02031CD72AD9
:10255000831605118312051102308316E8008312D9
:1025600038088316EA00831237088316E9008312BD
:102570003A088316EC00831239088316EB000A121E
:102580008A15831256220A168A1102308316DC003D
:10259000FA30831203179F000A1203134A220A1605
:1025A0008316DC0BC82A02308312CA00272B480886
:1025B0003002031CFF2A031DE12A2F0847020318DB
:1025C000FF2AC1080319F72A831605118312051182
:1025D00002308316DC00FA30831203179F000A12C0
:1025E00003134A220A168316DC0BEB2A8312C1015D
:1025F0000130C2008316851183128515272B300800
:102600004802031C272B031D092B47082F02031820
:10261000272BC20803191F2B8316851183128511DE
:1026200002308316DC00FA30831203179F000A126F
:1026300003134A220A168316DC0B132B8312013074
:10264000C100C2018316051183120515272B8316BD
:102650000C148312490B1C2C83168C120A30831223
:1026600033078316DC00831234088316DD00031859
:10267000DD0A03105C0DDE005D0DDF0083124F08E4
:1026800083165E078312C50083165F088312C60097
:1026900050080318500FC6070A128A1582230A161B
:1026A0008A11C00803198D2B32084602031C8D2B9A
:1026B000031D5E2B31084502031C8D2B831605106C
:1026C0008312051002308316E8008312380883163F
:1026D000EA00831237088316E90083123A0883164A
:1026E000EC00831239088316EB000A128A15831254
:1026F00056220A168A1102308316DC00FA30831241
:1027000003179F000A1203134A220A168316DC0BD2
:102710007E2B02308312C900192CBF080319C92B64
:1027200046083202031CC92B031D9A2B45083102AF
:10273000031CC92B83168510831285100230831663
:10274000E800831238088316EA00831237088316DC
:10275000E90083123A088316EC00831239088316C5
:10276000EB000A128A15831256220A168A110230C9
:102770008316DC00FA30831203179F000A1203133A
:102780004A220A168316DC0BBA2B02308312C900C8
:10279000192C46083202031CF12B031DD32B3108E0
:1027A00045020318F12BBF080319E92B8316851086
:1027B0008312851002308316DC00FA30831203176F
:1027C0009F000A1203134A220A168316DC0BDD2B24
:1027D0008312BF010130C000831605108312051457
:1027E000192C32084602031C192C031DFB2B45082B
:1027F00031020318192CC0080319112C8316051077
:102800008312051002308316DC00FA30831203179E
:102810009F000A1203134A220A168316DC0B052CAA
:1028200083120130BF00C001831685108312851406
:10283000192C83160C1483124A084904023C031D08
:102840006B2C02308316DC00FA30831203179F00D2
:102850000A1203134A220A168316DC0B242C0A12CE
:102860008A15831282230A168A1102308316E40025
:10287000831232088316E600831231088316E500BE
:102880000A128312D4230A16BF01C001C9013808F5
:10289000B4003708B30004308316E4008312300814
:1028A0008316E60083122F088316E5000A128312AE
:1028B000D4230A16C101C201CA013A08B600390878
:1028C000B500CC01CB01C3018316A0010C108C16FE
:1028D000C03083128B04071C732C871D732C871E3A
:1028E000732C071A782C0A128A15F42D0A168A11ED
:1028F00002308316E800831238088316EA00831238
:1029000037088316E90083123A088316EC00831215
:1029100039088316EB000A128A15831256220A160A
:062920008A11EB2963009F
:104204000300E8000300E8000000000000000000D4
:02400E00723FFF
:00000001FF
